:1000100083160030860003308500831285183A2845
:100020001128013086002C20023086002C2004305C
:1000300086002C20083086002C20103086002C20D2
:10004000203086002C20403086002C208030860016
:100050002C2085183A28112802308D0055308E004A
:10006000F0308F0064008F0B33288E0B30288D0BFF
:100070002E280800051C3A28013086002C20051C7B
:100080003F28023086002C20051C442804308600BE
:100090002C20051C4928083086002C20051C4E28E1
:1000A000103086002C20051C5328203086002C2080
:1000B000051C5828403086002C20051C5D28803007
:0A00C00086002C20051C62283A2857
:00000001FF
